Component: ARM Compiler 5.06 update 4 (build 422) Tool: armlink [4d35d2]

==============================================================================

Section Cross References

    clk.o(i.CLK_EnablePLL) refers to aeabi_sdiv.o(.text) for __aeabi_uidivmod
    clk.o(i.CLK_EnablePLL) refers to clk.o(i.CLK_WaitClockReady) for CLK_WaitClockReady
    clk.o(i.CLK_EnablePLL) refers to clk.o(i.CLK_GetPLLClockFreq) for CLK_GetPLLClockFreq
    clk.o(i.CLK_EnablePLL) refers to clk.o(.constdata) for .constdata
    clk.o(i.CLK_EnableXtalRC) refers to clk.o(i.CLK_WaitClockReady) for CLK_WaitClockReady
    clk.o(i.CLK_GetCPUFreq) refers to system_nano100series.o(i.SystemCoreClockUpdate) for SystemCoreClockUpdate
    clk.o(i.CLK_GetCPUFreq) refers to system_nano100series.o(.data) for SystemCoreClock
    clk.o(i.CLK_GetHCLKFreq) refers to system_nano100series.o(i.SystemCoreClockUpdate) for SystemCoreClockUpdate
    clk.o(i.CLK_GetHCLKFreq) refers to system_nano100series.o(.data) for SystemCoreClock
    clk.o(i.CLK_GetPLLClockFreq) refers to aeabi_sdiv.o(.text) for __aeabi_uidivmod
    clk.o(i.CLK_SetCoreClock) refers to clk.o(i.CLK_EnableXtalRC) for CLK_EnableXtalRC
    clk.o(i.CLK_SetCoreClock) refers to clk.o(i.CLK_SetHCLK) for CLK_SetHCLK
    clk.o(i.CLK_SetCoreClock) refers to clk.o(i.CLK_EnablePLL) for CLK_EnablePLL
    clk.o(i.CLK_SetCoreClock) refers to system_nano100series.o(.data) for SystemCoreClock
    clk.o(i.CLK_SetHCLK) refers to clk.o(i.CLK_WaitClockReady) for CLK_WaitClockReady
    clk.o(i.CLK_SetHCLK) refers to system_nano100series.o(i.SystemCoreClockUpdate) for SystemCoreClockUpdate
    clk.o(i.CLK_SysTickDelay) refers to system_nano100series.o(.data) for CyclesPerUs
    retarget.o(.emb_text) refers to retarget.o(i.Hard_Fault_Handler) for Hard_Fault_Handler
==============================================================================

Removing Unused input sections from the image.

    Removing clk.o(.rev16_text), (4 bytes).
    Removing clk.o(.revsh_text), (4 bytes).
    Removing clk.o(i.CLK_DisableCKO), (20 bytes).
    Removing clk.o(i.CLK_DisableModuleClock), (36 bytes).
    Removing clk.o(i.CLK_DisablePLL), (20 bytes).
    Removing clk.o(i.CLK_DisableSysTick), (12 bytes).
    Removing clk.o(i.CLK_DisableXtalRC), (16 bytes).
    Removing clk.o(i.CLK_EnableCKO), (40 bytes).
    Removing clk.o(i.CLK_EnablePLL), (224 bytes).
    Removing clk.o(i.CLK_EnableSysTick), (64 bytes).
    Removing clk.o(i.CLK_GetCPUFreq), (16 bytes).
    Removing clk.o(i.CLK_GetHCLKFreq), (16 bytes).
    Removing clk.o(i.CLK_GetHXTFreq), (28 bytes).
    Removing clk.o(i.CLK_GetLXTFreq), (24 bytes).
    Removing clk.o(i.CLK_GetPLLClockFreq), (128 bytes).
    Removing clk.o(i.CLK_Idle), (20 bytes).
    Removing clk.o(i.CLK_PowerDown), (32 bytes).
    Removing clk.o(i.CLK_SetCoreClock), (148 bytes).
==============================================================================

Image Symbol Table

    Local Symbols

    Symbol Name                              Value     Ov Type        Size  Object(Section)

    RESET                                    0x00000000   Section      192  startup_nano100series.o(RESET)
    ../clib/angel/boardlib.s                 0x00000000   Number         0  boardshut.o ABSOLUTE
    ../clib/angel/boardlib.s                 0x00000000   Number         0  boardinit3.o ABSOLUTE
    ../clib/angel/boardlib.s                 0x00000000   Number         0  boardinit2.o ABSOLUTE
    ../clib/angel/boardlib.s                 0x00000000   Number         0  boardinit1.o ABSOLUTE
    ../clib/angel/handlers.s                 0x00000000   Number         0  __scatter_zi.o ABSOLUTE
    ../clib/angel/handlers.s                 0x00000000   Number         0  __scatter_copy.o ABSOLUTE
    ../clib/angel/kernel.s                   0x00000000   Number         0  rtexit2.o ABSOLUTE
    ../clib/angel/kernel.s                   0x00000000   Number         0  rtexit.o ABSOLUTE
    ../clib/angel/kernel.s                   0x00000000   Number         0  __rtentry.o ABSOLUTE
    ../clib/angel/kernel.s                   0x00000000   Number         0  __rtentry2.o ABSOLUTE
    ../clib/angel/kernel.s                   0x00000000   Number         0  __rtentry4.o ABSOLUTE
    ../clib/angel/rt.s                       0x00000000   Number         0  aeabi_idiv0.o ABSOLUTE
    ../clib/angel/rt.s                       0x00000000   Number         0  aeabi_ldiv0_sigfpe.o ABSOLUTE
    ../clib/angel/rt.s                       0x00000000   Number         0  rt_locale.o ABSOLUTE
    ../clib/angel/rt.s                       0x00000000   Number         0  aeabi_ldiv0.o ABSOLUTE
    ../clib/angel/rt.s                       0x00000000   Number         0  rt_div0.o ABSOLUTE
    ../clib/angel/rt.s                       0x00000000   Number         0  rt_locale_intlibspace.o ABSOLUTE
    ../clib/angel/rt.s                       0x00000000   Number         0  rt_raise.o ABSOLUTE
    ../clib/angel/rt.s                       0x00000000   Number         0  aeabi_idiv0_sigfpe.o ABSOLUTE
    ../clib/angel/scatterp.s                 0x00000000   Number         0  __scatter.o ABSOLUTE
    ../clib/angel/startup.s                  0x00000000   Number         0  __main.o ABSOLUTE
    ../clib/angel/sys.s                      0x00000000   Number         0  indicate_semi.o ABSOLUTE
    ../clib/angel/sys.s                      0x00000000   Number         0  use_no_semi.o ABSOLUTE
    ../clib/angel/sys.s                      0x00000000   Number         0  tempstk.o ABSOLUTE
    ../clib/angel/sys.s                      0x00000000   Number         0  libspace.o ABSOLUTE
    ../clib/angel/sys.s                      0x00000000   Number         0  sys_stackheap_outer.o ABSOLUTE
    ../clib/angel/sysapp.c                   0x00000000   Number         0  sys_exit.o ABSOLUTE
    ../clib/angel/sysapp.c                   0x00000000   Number         0  sys_command.o ABSOLUTE
    ../clib/armsys.c                         0x00000000   Number         0  argv_veneer.o ABSOLUTE
    ../clib/armsys.c                         0x00000000   Number         0  no_argv.o ABSOLUTE
    ../clib/armsys.c                         0x00000000   Number         0  _get_argv_nomalloc.o ABSOLUTE
    ../clib/bigflt.c                         0x00000000   Number         0  bigflt0.o ABSOLUTE
    ../clib/btod.c                           0x00000000   Number         0  btod.o ABSOLUTE
    ../clib/division.c                       0x00000000   Number         0  lludiv10.o ABSOLUTE
    ../clib/division.c                       0x00000000   Number         0  lludiv.o ABSOLUTE
    ../clib/division.c                       0x00000000   Number         0  rtudiv10.o ABSOLUTE
    ../clib/division.c                       0x00000000   Number         0  llsdiv.o ABSOLUTE
    ../clib/division.s                       0x00000000   Number         0  aeabi_sdiv_div0.o ABSOLUTE
    ../clib/division.s                       0x00000000   Number         0  aeabi_sdiv.o ABSOLUTE
    ../clib/heapalloc.c                      0x00000000   Number         0  hrguard.o ABSOLUTE
    ../clib/heapaux.c                        0x00000000   Number         0  heapauxi.o ABSOLUTE
    ../clib/libinit.s                        0x00000000   Number         0  libinit.o ABSOLUTE
    ../clib/libinit.s                        0x00000000   Number         0  libinit2.o ABSOLUTE
    ../clib/libinit.s                        0x00000000   Number         0  libshutdown.o ABSOLUTE
    ../clib/libinit.s                        0x00000000   Number         0  libshutdown2.o ABSOLUTE
    ../clib/locale.s                         0x00000000   Number         0  lc_numeric_c.o ABSOLUTE
    ../clib/misc.s                           0x00000000   Number         0  printf_stubs.o ABSOLUTE
    ../clib/printf.c                         0x00000000   Number         0  _printf_hex_int.o ABSOLUTE
    ../clib/printf.c                         0x00000000   Number         0  __printf_ss.o ABSOLUTE
    ../clib/printf.c                         0x00000000   Number         0  _printf_hex_int_ptr.o ABSOLUTE
    ../clib/printf.c                         0x00000000   Number         0  _printf_hex_ptr.o ABSOLUTE
    ../clib/printf.c                         0x00000000   Number         0  __printf_flags_ss.o ABSOLUTE
    ../clib/printf.c                         0x00000000   Number         0  __printf_wp.o ABSOLUTE
    ../clib/printf.c                         0x00000000   Number         0  _printf_hex_int_ll.o ABSOLUTE
    ../clib/printf.c                         0x00000000   Number         0  __printf_flags_wp.o ABSOLUTE
    ../clib/printf.c                         0x00000000   Number         0  _printf_fp_dec.o ABSOLUTE
    ../clib/printf.c                         0x00000000   Number         0  __printf_ss_wp.o ABSOLUTE
    ../clib/printf.c                         0x00000000   Number         0  __printf_flags_ss_wp.o ABSOLUTE
    ../clib/printf.c                         0x00000000   Number         0  __2printf.o ABSOLUTE
    ../clib/printf.c                         0x00000000   Number         0  __2sprintf.o ABSOLUTE
    ../clib/printf.c                         0x00000000   Number         0  noretval__2printf.o ABSOLUTE
    ../clib/printf.c                         0x00000000   Number         0  _printf_fp_infnan.o ABSOLUTE
    ../clib/printf.c                         0x00000000   Number         0  __printf_nopercent.o ABSOLUTE
    ../clib/printf.c                         0x00000000   Number         0  __printf.o ABSOLUTE
    ../clib/printf.c                         0x00000000   Number         0  _printf_pad.o ABSOLUTE
    ../clib/printf.c                         0x00000000   Number         0  _printf_str.o ABSOLUTE
    ../clib/printf.c                         0x00000000   Number         0  _sputc.o ABSOLUTE
    ../clib/printf.c                         0x00000000   Number         0  _printf_intcommon.o ABSOLUTE
    ../clib/printf.c                         0x00000000   Number         0  _printf_char_common.o ABSOLUTE
    ../clib/printf.c                         0x00000000   Number         0  _printf_dec.o ABSOLUTE
    ../clib/printf.c                         0x00000000   Number         0  _printf_char.o ABSOLUTE
    ../clib/printf.c                         0x00000000   Number         0  __printf_flags.o ABSOLUTE
    ../clib/printf.c                         0x00000000   Number         0  _printf_hex_ll.o ABSOLUTE
    ../clib/printf.c                         0x00000000   Number         0  _printf_hex_int_ll_ptr.o ABSOLUTE
    ../clib/printf.c                         0x00000000   Number         0  _printf_hex_ll_ptr.o ABSOLUTE
    ../clib/printf.c                         0x00000000   Number         0  _printf_char_file.o ABSOLUTE
    ../clib/printf.c                         0x00000000   Number         0  noretval__2sprintf.o ABSOLUTE
    ../clib/printf_percent.s                 0x00000000   Number         0  _printf_d.o ABSOLUTE
    ../clib/printf_percent.s                 0x00000000   Number         0  _printf_s.o ABSOLUTE
    ../clib/printf_percent.s                 0x00000000   Number         0  _printf_f.o ABSOLUTE
    ../clib/printf_percent.s                 0x00000000   Number         0  _printf_percent.o ABSOLUTE
    ../clib/printf_percent.s                 0x00000000   Number         0  _printf_percent_end.o ABSOLUTE
    ../clib/printf_percent.s                 0x00000000   Number         0  _printf_x.o ABSOLUTE
    ../clib/signal.c                         0x00000000   Number         0  __raise.o ABSOLUTE
    ../clib/signal.c                         0x00000000   Number         0  defsig_fpe_inner.o ABSOLUTE
    ../clib/signal.c                         0x00000000   Number         0  defsig_rtmem_formal.o ABSOLUTE
    ../clib/signal.c                         0x00000000   Number         0  defsig_exit.o ABSOLUTE
    ../clib/signal.c                         0x00000000   Number         0  defsig_fpe_formal.o ABSOLUTE
    ../clib/signal.c                         0x00000000   Number         0  defsig_abrt_inner.o ABSOLUTE
    ../clib/signal.c                         0x00000000   Number         0  defsig_rtred_inner.o ABSOLUTE
    ../clib/signal.c                         0x00000000   Number         0  defsig_rtmem_inner.o ABSOLUTE
    ../clib/signal.c                         0x00000000   Number         0  defsig_stak_inner.o ABSOLUTE
    ../clib/signal.c                         0x00000000   Number         0  defsig_pvfn_inner.o ABSOLUTE
    ../clib/signal.c                         0x00000000   Number         0  defsig_cppl_inner.o ABSOLUTE
    ../clib/signal.c                         0x00000000   Number         0  defsig_segv_inner.o ABSOLUTE
    ../clib/signal.c                         0x00000000   Number         0  defsig_other.o ABSOLUTE
    ../clib/signal.c                         0x00000000   Number         0  defsig_fpe_outer.o ABSOLUTE
    ../clib/signal.c                         0x00000000   Number         0  defsig_rtmem_outer.o ABSOLUTE
    ../clib/signal.c                         0x00000000   Number         0  defsig_general.o ABSOLUTE
    ../clib/signal.s                         0x00000000   Number         0  defsig.o ABSOLUTE
    ../clib/stdlib.c                         0x00000000   Number         0  exit.o ABSOLUTE
    ../clib/string.c                         0x00000000   Number         0  strlen.o ABSOLUTE
    ../clib/string.c                         0x00000000   Number         0  strcmp.o ABSOLUTE
    ../fplib/cfplib/f2d.c                    0x00000000   Number         0  f2d.o ABSOLUTE
    ../fplib/cfplib/fdiv.c                   0x00000000   Number         0  fdiv.o ABSOLUTE
    ../fplib/cfplib/fflt.c                   0x00000000   Number         0  fflti.o ABSOLUTE
    ../fplib/cfplib/fpinit.c                 0x00000000   Number         0  fpinit.o ABSOLUTE
    ../fplib/cfplib/ieee_status.c            0x00000000   Number         0  ieee_status.o ABSOLUTE
    ../fplib/printf1.s                       0x00000000   Number         0  printf1.o ABSOLUTE
    ../fplib/usenofp.s                       0x00000000   Number         0  usenofp.o ABSOLUTE
    ../mathlib/fpclassify.c                  0x00000000   Number         0  fpclassify.o ABSOLUTE
    ..\\nuvoton\\nuvoton\\Library\\Device\\Nuvoton\\Nano100Series\\Source\\system_Nano100Series.c 0x00000000   Number         0  system_nano100series.o ABSOLUTE
    ..\\nuvoton\\nuvoton\\Library\\StdDriver\\src\\clk.c 0x00000000   Number         0  clk.o ABSOLUTE
    ..\\nuvoton\\nuvoton\\Library\\StdDriver\\src\\gpio.c 0x00000000   Number         0  gpio.o ABSOLUTE
    ..\\nuvoton\\nuvoton\\Library\\StdDriver\\src\\retarget.c 0x00000000   Number         0  retarget.o ABSOLUTE
    ..\\nuvoton\\nuvoton\\Library\\StdDriver\\src\\sys.c 0x00000000   Number         0  sys.o ABSOLUTE
    ..\\nuvoton\\nuvoton\\Library\\StdDriver\\src\\timer.c 0x00000000   Number         0  timer.o ABSOLUTE
    ..\\nuvoton\\nuvoton\\Library\\StdDriver\\src\\uart.c 0x00000000   Number         0  uart.o ABSOLUTE
    ..\nuvoton\nuvoton\Library\Device\Nuvoton\Nano100Series\Source\ARM\startup_Nano100Series.s 0x00000000   Number         0  startup_nano100series.o ABSOLUTE
    ..\nuvoton\nuvoton\Library\Device\Nuvoton\Nano100Series\Source\system_Nano100Series.c 0x00000000   Number         0  system_nano100series.o ABSOLUTE
    ..\nuvoton\nuvoton\Library\StdDriver\src\clk.c 0x00000000   Number         0  clk.o ABSOLUTE
    ..\nuvoton\nuvoton\Library\StdDriver\src\gpio.c 0x00000000   Number         0  gpio.o ABSOLUTE
    ..\nuvoton\nuvoton\Library\StdDriver\src\retarget.c 0x00000000   Number         0  retarget.o ABSOLUTE
    ..\nuvoton\nuvoton\Library\StdDriver\src\sys.c 0x00000000   Number         0  sys.o ABSOLUTE
    ..\nuvoton\nuvoton\Library\StdDriver\src\timer.c 0x00000000   Number         0  timer.o ABSOLUTE
    ..\nuvoton\nuvoton\Library\StdDriver\src\uart.c 0x00000000   Number         0  uart.o ABSOLUTE
    dc.s                                     0x00000000   Number         0  dc.o ABSOLUTE
    main.c                                   0x00000000   Number         0  main.o ABSOLUTE
    main.c                                   0x00000000   Number         0  main.o ABSOLUTE
    !!!main                                  0x000000c0   Section        8  __main.o(!!!main)
    !!!scatter                               0x000000c8   Section       60  __scatter.o(!!!scatter)
    !!handler_copy                           0x00000104   Section       26  __scatter_copy.o(!!handler_copy)
    !!handler_zi                             0x00000120   Section       28  __scatter_zi.o(!!handler_zi)
    .ARM.Collect$$_printf_percent$$00000000  0x0000013c   Section        2  _printf_percent.o(.ARM.Collect$$_printf_percent$$00000000)
    .ARM.Collect$$_printf_percent$$00000009  0x0000013e   Section       10  _printf_d.o(.ARM.Collect$$_printf_percent$$00000009)
    .ARM.Collect$$_printf_percent$$0000000C  0x00000148   Section       10  _printf_x.o(.ARM.Collect$$_printf_percent$$0000000C)
    .ARM.Collect$$_printf_percent$$00000014  0x00000152   Section       10  _printf_s.o(.ARM.Collect$$_printf_percent$$00000014)
    .ARM.Collect$$_printf_percent$$00000017  0x0000015c   Section        4  _printf_percent_end.o(.ARM.Collect$$_printf_percent$$00000017)
    .ARM.Collect$$libinit$$00000000          0x00000160   Section        2  libinit.o(.ARM.Collect$$libinit$$00000000)
    .ARM.Collect$$libinit$$00000002          0x00000162   Section        0  libinit2.o(.ARM.Collect$$libinit$$00000002)
    .ARM.Collect$$libinit$$00000004          0x00000162   Section        0  libinit2.o(.ARM.Collect$$libinit$$00000004)
    .ARM.Collect$$libinit$$0000000A          0x00000162   Section        0  libinit2.o(.ARM.Collect$$libinit$$0000000A)
    .ARM.Collect$$libinit$$0000000C          0x00000162   Section        0  libinit2.o(.ARM.Collect$$libinit$$0000000C)
    .ARM.Collect$$libinit$$0000000E          0x00000162   Section        0  libinit2.o(.ARM.Collect$$libinit$$0000000E)
    .ARM.Collect$$libinit$$00000011          0x00000162   Section        0  libinit2.o(.ARM.Collect$$libinit$$00000011)
    .ARM.Collect$$libinit$$00000013          0x00000162   Section        0  libinit2.o(.ARM.Collect$$libinit$$00000013)
    .ARM.Collect$$libinit$$00000015          0x00000162   Section        0  libinit2.o(.ARM.Collect$$libinit$$00000015)
    .ARM.Collect$$libinit$$00000017          0x00000162   Section        0  libinit2.o(.ARM.Collect$$libinit$$00000017)
    .ARM.Collect$$libinit$$00000019          0x00000162   Section        0  libinit2.o(.ARM.Collect$$libinit$$00000019)
    .ARM.Collect$$libinit$$0000001B          0x00000162   Section        0  libinit2.o(.ARM.Collect$$libinit$$0000001B)
    .ARM.Collect$$libinit$$0000001D          0x00000162   Section        0  libinit2.o(.ARM.Collect$$libinit$$0000001D)
    .ARM.Collect$$libinit$$0000001F          0x00000162   Section        0  libinit2.o(.ARM.Collect$$libinit$$0000001F)
    .ARM.Collect$$libinit$$00000021          0x00000162   Section        0  libinit2.o(.ARM.Collect$$libinit$$00000021)
    .ARM.Collect$$libinit$$00000023          0x00000162   Section        0  libinit2.o(.ARM.Collect$$libinit$$00000023)
    .ARM.Collect$$libinit$$00000025          0x00000162   Section        0  libinit2.o(.ARM.Collect$$libinit$$00000025)
    .ARM.Collect$$libinit$$0000002C          0x00000162   Section        0  libinit2.o(.ARM.Collect$$libinit$$0000002C)
    .ARM.Collect$$libinit$$0000002E          0x00000162   Section        0  libinit2.o(.ARM.Collect$$libinit$$0000002E)
    .ARM.Collect$$libinit$$00000030          0x00000162   Section        0  libinit2.o(.ARM.Collect$$libinit$$00000030)
    .ARM.Collect$$libinit$$00000032          0x00000162   Section        0  libinit2.o(.ARM.Collect$$libinit$$00000032)
    .ARM.Collect$$libinit$$00000033          0x00000162   Section        2  libinit2.o(.ARM.Collect$$libinit$$00000033)
    .ARM.Collect$$libshutdown$$00000000      0x00000164   Section        2  libshutdown.o(.ARM.Collect$$libshutdown$$00000000)
    .ARM.Collect$$libshutdown$$00000002      0x00000166   Section        0  libshutdown2.o(.ARM.Collect$$libshutdown$$00000002)
    .ARM.Collect$$libshutdown$$00000004      0x00000166   Section        0  libshutdown2.o(.ARM.Collect$$libshutdown$$00000004)
    .ARM.Collect$$libshutdown$$00000007      0x00000166   Section        0  libshutdown2.o(.ARM.Collect$$libshutdown$$00000007)
    .ARM.Collect$$libshutdown$$0000000A      0x00000166   Section        0  libshutdown2.o(.ARM.Collect$$libshutdown$$0000000A)
    .ARM.Collect$$libshutdown$$0000000C      0x00000166   Section        0  libshutdown2.o(.ARM.Collect$$libshutdown$$0000000C)
    .ARM.Collect$$libshutdown$$0000000F      0x00000166   Section        0  libshutdown2.o(.ARM.Collect$$libshutdown$$0000000F)
    .ARM.Collect$$libshutdown$$00000010      0x00000166   Section        2  libshutdown2.o(.ARM.Collect$$libshutdown$$00000010)
    .ARM.Collect$$rtentry$$00000000          0x00000168   Section        0  __rtentry.o(.ARM.Collect$$rtentry$$00000000)
    .ARM.Collect$$rtentry$$00000002          0x00000168   Section        0  __rtentry2.o(.ARM.Collect$$rtentry$$00000002)
    .ARM.Collect$$rtentry$$00000004          0x00000168   Section        6  __rtentry4.o(.ARM.Collect$$rtentry$$00000004)
    .ARM.Collect$$rtentry$$00000009          0x0000016e   Section        0  __rtentry2.o(.ARM.Collect$$rtentry$$00000009)
    .ARM.Collect$$rtentry$$0000000A          0x0000016e   Section        4  __rtentry2.o(.ARM.Collect$$rtentry$$0000000A)
    .ARM.Collect$$rtentry$$0000000C          0x00000172   Section        0  __rtentry2.o(.ARM.Collect$$rtentry$$0000000C)
    .ARM.Collect$$rtentry$$0000000D          0x00000172   Section        8  __rtentry2.o(.ARM.Collect$$rtentry$$0000000D)
    .ARM.Collect$$rtexit$$00000000           0x0000017a   Section        2  rtexit.o(.ARM.Collect$$rtexit$$00000000)
    .ARM.Collect$$rtexit$$00000002           0x0000017c   Section        0  rtexit2.o(.ARM.Collect$$rtexit$$00000002)
    .ARM.Collect$$rtexit$$00000003           0x0000017c   Section        4  rtexit2.o(.ARM.Collect$$rtexit$$00000003)
    .ARM.Collect$$rtexit$$00000004           0x00000180   Section        6  rtexit2.o(.ARM.Collect$$rtexit$$00000004)
    .emb_text                                0x00000188   Section       28  retarget.o(.emb_text)
    .text                                    0x000001a4   Section       96  startup_nano100series.o(.text)
    .text                                    0x00000204   Section        0  llsdiv.o(.text)
    .text                                    0x00000274   Section        0  noretval__2printf.o(.text)
    .text                                    0x00000290   Section        0  noretval__2sprintf.o(.text)
    .text                                    0x000002b8   Section        0  _printf_pad.o(.text)
    .text                                    0x00000306   Section        0  _printf_str.o(.text)
    .text                                    0x00000358   Section        0  _printf_dec.o(.text)
    .text                                    0x000003c4   Section        0  _printf_hex_int.o(.text)
    .text                                    0x0000041c   Section        0  __printf_flags_wp.o(.text)
    .text                                    0x00000554   Section        0  strlen.o(.text)
    .text                                    0x00000598   Section      346  aeabi_sdiv.o(.text)
    .text                                    0x000006f2   Section        0  heapauxi.o(.text)
    .text                                    0x000006f8   Section        0  lludiv.o(.text)
    .text                                    0x000007fa   Section        0  _printf_intcommon.o(.text)
    .text                                    0x000008ac   Section        0  _printf_char_common.o(.text)
    _printf_input_char                       0x000008ad   Thumb Code    10  _printf_char_common.o(.text)
    .text                                    0x000008dc   Section        0  _sputc.o(.text)
    .text                                    0x000008e6   Section        0  _printf_char.o(.text)
    .text                                    0x00000914   Section        0  _printf_char_file.o(.text)
    .text                                    0x0000093c   Section        0  rtudiv10.o(.text)
    .text                                    0x00000964   Section        8  libspace.o(.text)
    .text                                    0x0000096c   Section       62  sys_stackheap_outer.o(.text)
    .text                                    0x000009aa   Section        0  exit.o(.text)
    .text                                    0x000009bc   Section        0  sys_exit.o(.text)
    .text                                    0x000009c8   Section        2  use_no_semi.o(.text)
    .text                                    0x000009ca   Section        0  indicate_semi.o(.text)
    i.CLK_EnableModuleClock                  0x000009cc   Section        0  clk.o(i.CLK_EnableModuleClock)
    i.CLK_EnableXtalRC                       0x000009f0   Section        0  clk.o(i.CLK_EnableXtalRC)
    i.CLK_SetHCLK                            0x00000a3c   Section        0  clk.o(i.CLK_SetHCLK)
    i.CLK_SetModuleClock                     0x00000aa0   Section        0  clk.o(i.CLK_SetModuleClock)
    i.CLK_WaitClockReady                     0x00000b04   Section        0  clk.o(i.CLK_WaitClockReady)
    i.GPIO_SetMode                           0x00000b2c   Section        0  gpio.o(i.GPIO_SetMode)
    i.Hard_Fault_Handler                     0x00000b5c   Section        0  retarget.o(i.Hard_Fault_Handler)
    __tagsym$$used                           0x00000b5d   Number         0  retarget.o(i.Hard_Fault_Handler)
    i.SendChar                               0x00000b88   Section        0  retarget.o(i.SendChar)
    i.SendChar_ToUART                        0x00000b94   Section        0  retarget.o(i.SendChar_ToUART)
    i.SysGet_HCLKFreq                        0x00000bc8   Section        0  system_nano100series.o(i.SysGet_HCLKFreq)
    i.SysGet_PLLClockFreq                    0x00000c18   Section        0  system_nano100series.o(i.SysGet_PLLClockFreq)
    i.SystemCoreClockUpdate                  0x00000c98   Section        0  system_nano100series.o(i.SystemCoreClockUpdate)
    i.TIMER_Delay                            0x00000cc4   Section        0  timer.o(i.TIMER_Delay)
    i.TIMER_GetModuleClock                   0x00000d78   Section        0  timer.o(i.TIMER_GetModuleClock)
    i.UART1_IRQHandler                       0x00000df8   Section        0  main.o(i.UART1_IRQHandler)
    i.UART_ClearIntFlag                      0x00000e14   Section        0  uart.o(i.UART_ClearIntFlag)
    i.UART_EnableInt                         0x00000e84   Section        0  uart.o(i.UART_EnableInt)
    i.UART_Open                              0x00000e8c   Section        0  uart.o(i.UART_Open)
    i.UART_Write                             0x00000f2c   Section        0  uart.o(i.UART_Write)
    i.__ARM_common_ll_muluu                  0x00000f62   Section        0  timer.o(i.__ARM_common_ll_muluu)
    i._is_digit                              0x00000f92   Section        0  __printf_wp.o(i._is_digit)
    i.ferror                                 0x00000fa0   Section        0  retarget.o(i.ferror)
    i.fputc                                  0x00000fa8   Section        0  retarget.o(i.fputc)
    i.init                                   0x00000fb8   Section        0  main.o(i.init)
    i.main                                   0x00001080   Section        0  main.o(i.main)
    i.stackDump                              0x000011fc   Section        0  retarget.o(i.stackDump)
    .constdata                               0x000012a4   Section       16  timer.o(.constdata)
    .constdata                               0x000012b4   Section       48  uart.o(.constdata)
    .constdata                               0x000012e4   Section       40  _printf_hex_int.o(.constdata)
    uc_hextab                                0x000012e4   Data          20  _printf_hex_int.o(.constdata)
    lc_hextab                                0x000012f8   Data          20  _printf_hex_int.o(.constdata)
    .constdata                               0x0000130c   Section       17  __printf_flags_wp.o(.constdata)
    maptable                                 0x0000130c   Data          17  __printf_flags_wp.o(.constdata)
    .conststring                             0x00001320   Section       67  main.o(.conststring)
    .data                                    0x20000000   Section        8  retarget.o(.data)
    .data                                    0x20000008   Section        8  system_nano100series.o(.data)
    .bss                                     0x20000010   Section       96  libspace.o(.bss)
    HEAP                                     0x20000070   Section     1280  startup_nano100series.o(HEAP)
    Heap_Mem                                 0x20000070   Data        1280  startup_nano100series.o(HEAP)
    STACK                                    0x20000570   Section     1280  startup_nano100series.o(STACK)
    Stack_Mem                                0x20000570   Data        1280  startup_nano100series.o(STACK)
    __initial_sp                             0x20000a70   Data           0  startup_nano100series.o(STACK)

    Global Symbols

    Symbol Name                              Value     Ov Type        Size  Object(Section)

    BuildAttributes$$THM_ISAv3M$S$PE$A:L22$X:L11$S22$IEEE1$IW$USESV6$~STKCKD$USESV7$~SHL$OTIME$ROPI$IEEEJ$EBA8$UX$STANDARDLIB$REQ8$PRES8$EABIv2 0x00000000   Number         0  anon$$obj.o ABSOLUTE
    __ARM_use_no_argv                        0x00000000   Number         0  main.o ABSOLUTE
    __Vectors                                0x00000000   Data           4  startup_nano100series.o(RESET)
    _printf_flags                            0x00000000   Number         0  printf_stubs.o ABSOLUTE
    _printf_return_value                     0x00000000   Number         0  printf_stubs.o ABSOLUTE
    _printf_sizespec                         0x00000000   Number         0  printf_stubs.o ABSOLUTE
    _printf_widthprec                        0x00000000   Number         0  printf_stubs.o ABSOLUTE
    __ARM_exceptions_init                     - Undefined Weak Reference
    __alloca_initialize                       - Undefined Weak Reference
    __arm_preinit_                            - Undefined Weak Reference
    __cpp_initialize__aeabi_                  - Undefined Weak Reference
    __cxa_finalize                            - Undefined Weak Reference
    __sigvec_lookup                           - Undefined Weak Reference
    _atexit_init                              - Undefined Weak Reference
    _call_atexit_fns                          - Undefined Weak Reference
    _clock_init                               - Undefined Weak Reference
    _fp_trap_init                             - Undefined Weak Reference
    _fp_trap_shutdown                         - Undefined Weak Reference
    _get_lc_collate                           - Undefined Weak Reference
    _get_lc_ctype                             - Undefined Weak Reference
    _get_lc_monetary                          - Undefined Weak Reference
    _get_lc_time                              - Undefined Weak Reference
    _getenv_init                              - Undefined Weak Reference
    _handle_redirection                       - Undefined Weak Reference
    _init_alloc                               - Undefined Weak Reference
    _init_user_alloc                          - Undefined Weak Reference
    _initio                                   - Undefined Weak Reference
    _printf_mbtowc                            - Undefined Weak Reference
    _printf_truncate_signed                   - Undefined Weak Reference
    _printf_truncate_unsigned                 - Undefined Weak Reference
    _rand_init                                - Undefined Weak Reference
    _signal_finish                            - Undefined Weak Reference
    _signal_init                              - Undefined Weak Reference
    _terminate_alloc                          - Undefined Weak Reference
    _terminate_user_alloc                     - Undefined Weak Reference
    _terminateio                              - Undefined Weak Reference
    __main                                   0x000000c1   Thumb Code     8  __main.o(!!!main)
    __scatterload                            0x000000c9   Thumb Code     0  __scatter.o(!!!scatter)
    __scatterload_rt2                        0x000000c9   Thumb Code    52  __scatter.o(!!!scatter)
    __scatterload_rt2_thumb_only             0x000000c9   Thumb Code     0  __scatter.o(!!!scatter)
    __scatterload_null                       0x000000d9   Thumb Code     0  __scatter.o(!!!scatter)
    __scatterload_copy                       0x00000105   Thumb Code    26  __scatter_copy.o(!!handler_copy)
    __scatterload_zeroinit                   0x00000121   Thumb Code    28  __scatter_zi.o(!!handler_zi)
    _printf_percent                          0x0000013d   Thumb Code     0  _printf_percent.o(.ARM.Collect$$_printf_percent$$00000000)
    _printf_d                                0x0000013f   Thumb Code     0  _printf_d.o(.ARM.Collect$$_printf_percent$$00000009)
    _printf_x                                0x00000149   Thumb Code     0  _printf_x.o(.ARM.Collect$$_printf_percent$$0000000C)
    _printf_s                                0x00000153   Thumb Code     0  _printf_s.o(.ARM.Collect$$_printf_percent$$00000014)
    _printf_percent_end                      0x0000015d   Thumb Code     0  _printf_percent_end.o(.ARM.Collect$$_printf_percent$$00000017)
    __rt_lib_init                            0x00000161   Thumb Code     0  libinit.o(.ARM.Collect$$libinit$$00000000)
    __rt_lib_init_alloca_1                   0x00000163   Thumb Code     0  libinit2.o(.ARM.Collect$$libinit$$0000002E)
    __rt_lib_init_argv_1                     0x00000163   Thumb Code     0  libinit2.o(.ARM.Collect$$libinit$$0000002C)
    __rt_lib_init_atexit_1                   0x00000163   Thumb Code     0  libinit2.o(.ARM.Collect$$libinit$$0000001B)
    __rt_lib_init_clock_1                    0x00000163   Thumb Code     0  libinit2.o(.ARM.Collect$$libinit$$00000021)
    __rt_lib_init_cpp_1                      0x00000163   Thumb Code     0  libinit2.o(.ARM.Collect$$libinit$$00000032)
    __rt_lib_init_exceptions_1               0x00000163   Thumb Code     0  libinit2.o(.ARM.Collect$$libinit$$00000030)
    __rt_lib_init_fp_1                       0x00000163   Thumb Code     0  libinit2.o(.ARM.Collect$$libinit$$00000002)
    __rt_lib_init_fp_trap_1                  0x00000163   Thumb Code     0  libinit2.o(.ARM.Collect$$libinit$$0000001F)
    __rt_lib_init_getenv_1                   0x00000163   Thumb Code     0  libinit2.o(.ARM.Collect$$libinit$$00000023)
    __rt_lib_init_heap_1                     0x00000163   Thumb Code     0  libinit2.o(.ARM.Collect$$libinit$$0000000A)
    __rt_lib_init_lc_collate_1               0x00000163   Thumb Code     0  libinit2.o(.ARM.Collect$$libinit$$00000011)
    __rt_lib_init_lc_ctype_1                 0x00000163   Thumb Code     0  libinit2.o(.ARM.Collect$$libinit$$00000013)
    __rt_lib_init_lc_monetary_1              0x00000163   Thumb Code     0  libinit2.o(.ARM.Collect$$libinit$$00000015)
    __rt_lib_init_lc_numeric_1               0x00000163   Thumb Code     0  libinit2.o(.ARM.Collect$$libinit$$00000017)
    __rt_lib_init_lc_time_1                  0x00000163   Thumb Code     0  libinit2.o(.ARM.Collect$$libinit$$00000019)
    __rt_lib_init_preinit_1                  0x00000163   Thumb Code     0  libinit2.o(.ARM.Collect$$libinit$$00000004)
    __rt_lib_init_rand_1                     0x00000163   Thumb Code     0  libinit2.o(.ARM.Collect$$libinit$$0000000E)
    __rt_lib_init_return                     0x00000163   Thumb Code     0  libinit2.o(.ARM.Collect$$libinit$$00000033)
    __rt_lib_init_signal_1                   0x00000163   Thumb Code     0  libinit2.o(.ARM.Collect$$libinit$$0000001D)
    __rt_lib_init_stdio_1                    0x00000163   Thumb Code     0  libinit2.o(.ARM.Collect$$libinit$$00000025)
    __rt_lib_init_user_alloc_1               0x00000163   Thumb Code     0  libinit2.o(.ARM.Collect$$libinit$$0000000C)
    __rt_lib_shutdown                        0x00000165   Thumb Code     0  libshutdown.o(.ARM.Collect$$libshutdown$$00000000)
    __rt_lib_shutdown_cpp_1                  0x00000167   Thumb Code     0  libshutdown2.o(.ARM.Collect$$libshutdown$$00000002)
    __rt_lib_shutdown_fp_trap_1              0x00000167   Thumb Code     0  libshutdown2.o(.ARM.Collect$$libshutdown$$00000007)
    __rt_lib_shutdown_heap_1                 0x00000167   Thumb Code     0  libshutdown2.o(.ARM.Collect$$libshutdown$$0000000F)
    __rt_lib_shutdown_return                 0x00000167   Thumb Code     0  libshutdown2.o(.ARM.Collect$$libshutdown$$00000010)
    __rt_lib_shutdown_signal_1               0x00000167   Thumb Code     0  libshutdown2.o(.ARM.Collect$$libshutdown$$0000000A)
    __rt_lib_shutdown_stdio_1                0x00000167   Thumb Code     0  libshutdown2.o(.ARM.Collect$$libshutdown$$00000004)
    __rt_lib_shutdown_user_alloc_1           0x00000167   Thumb Code     0  libshutdown2.o(.ARM.Collect$$libshutdown$$0000000C)
    __rt_entry                               0x00000169   Thumb Code     0  __rtentry.o(.ARM.Collect$$rtentry$$00000000)
    __rt_entry_presh_1                       0x00000169   Thumb Code     0  __rtentry2.o(.ARM.Collect$$rtentry$$00000002)
    __rt_entry_sh                            0x00000169   Thumb Code     0  __rtentry4.o(.ARM.Collect$$rtentry$$00000004)
    __rt_entry_li                            0x0000016f   Thumb Code     0  __rtentry2.o(.ARM.Collect$$rtentry$$0000000A)
    __rt_entry_postsh_1                      0x0000016f   Thumb Code     0  __rtentry2.o(.ARM.Collect$$rtentry$$00000009)
    __rt_entry_main                          0x00000173   Thumb Code     0  __rtentry2.o(.ARM.Collect$$rtentry$$0000000D)
    __rt_entry_postli_1                      0x00000173   Thumb Code     0  __rtentry2.o(.ARM.Collect$$rtentry$$0000000C)
    __rt_exit                                0x0000017b   Thumb Code     0  rtexit.o(.ARM.Collect$$rtexit$$00000000)
    __rt_exit_ls                             0x0000017d   Thumb Code     0  rtexit2.o(.ARM.Collect$$rtexit$$00000003)
    __rt_exit_prels_1                        0x0000017d   Thumb Code     0  rtexit2.o(.ARM.Collect$$rtexit$$00000002)
    __rt_exit_exit                           0x00000181   Thumb Code     0  rtexit2.o(.ARM.Collect$$rtexit$$00000004)
    HardFault_Handler                        0x00000189   Thumb Code    24  retarget.o(.emb_text)
    Reset_Handler                            0x000001a5   Thumb Code    28  startup_nano100series.o(.text)
    NMI_Handler                              0x000001c1   Thumb Code     2  startup_nano100series.o(.text)
    SVC_Handler                              0x000001c5   Thumb Code     2  startup_nano100series.o(.text)
    PendSV_Handler                           0x000001c7   Thumb Code     2  startup_nano100series.o(.text)
    SysTick_Handler                          0x000001c9   Thumb Code     2  startup_nano100series.o(.text)
    ADC_IRQHandler                           0x000001cb   Thumb Code     0  startup_nano100series.o(.text)
    BOD_IRQHandler                           0x000001cb   Thumb Code     0  startup_nano100series.o(.text)
    DAC_IRQHandler                           0x000001cb   Thumb Code     0  startup_nano100series.o(.text)
    EINT0_IRQHandler                         0x000001cb   Thumb Code     0  startup_nano100series.o(.text)
    EINT1_IRQHandler                         0x000001cb   Thumb Code     0  startup_nano100series.o(.text)
    GPABC_IRQHandler                         0x000001cb   Thumb Code     0  startup_nano100series.o(.text)
    GPDEF_IRQHandler                         0x000001cb   Thumb Code     0  startup_nano100series.o(.text)
    HIRC_IRQHandler                          0x000001cb   Thumb Code     0  startup_nano100series.o(.text)
    I2C0_IRQHandler                          0x000001cb   Thumb Code     0  startup_nano100series.o(.text)
    I2C1_IRQHandler                          0x000001cb   Thumb Code     0  startup_nano100series.o(.text)
    I2S_IRQHandler                           0x000001cb   Thumb Code     0  startup_nano100series.o(.text)
    LCD_IRQHandler                           0x000001cb   Thumb Code     0  startup_nano100series.o(.text)
    PDMA_IRQHandler                          0x000001cb   Thumb Code     0  startup_nano100series.o(.text)
    PDWU_IRQHandler                          0x000001cb   Thumb Code     0  startup_nano100series.o(.text)
    PWM0_IRQHandler                          0x000001cb   Thumb Code     0  startup_nano100series.o(.text)
    PWM1_IRQHandler                          0x000001cb   Thumb Code     0  startup_nano100series.o(.text)
    RTC_IRQHandler                           0x000001cb   Thumb Code     0  startup_nano100series.o(.text)
    SC0_IRQHandler                           0x000001cb   Thumb Code     0  startup_nano100series.o(.text)
    SC1_IRQHandler                           0x000001cb   Thumb Code     0  startup_nano100series.o(.text)
    SC2_IRQHandler                           0x000001cb   Thumb Code     0  startup_nano100series.o(.text)
    SPI0_IRQHandler                          0x000001cb   Thumb Code     0  startup_nano100series.o(.text)
    SPI1_IRQHandler                          0x000001cb   Thumb Code     0  startup_nano100series.o(.text)
    SPI2_IRQHandler                          0x000001cb   Thumb Code     0  startup_nano100series.o(.text)
    TMR0_IRQHandler                          0x000001cb   Thumb Code     0  startup_nano100series.o(.text)
    TMR1_IRQHandler                          0x000001cb   Thumb Code     0  startup_nano100series.o(.text)
    TMR2_IRQHandler                          0x000001cb   Thumb Code     0  startup_nano100series.o(.text)
    TMR3_IRQHandler                          0x000001cb   Thumb Code     0  startup_nano100series.o(.text)
    UART0_IRQHandler                         0x000001cb   Thumb Code     0  startup_nano100series.o(.text)
    USBD_IRQHandler                          0x000001cb   Thumb Code     0  startup_nano100series.o(.text)
    WDT_IRQHandler                           0x000001cb   Thumb Code     0  startup_nano100series.o(.text)
    __user_initial_stackheap                 0x000001cd   Thumb Code     0  startup_nano100series.o(.text)
    __aeabi_ldivmod                          0x00000205   Thumb Code   112  llsdiv.o(.text)
    _ll_sdiv                                 0x00000205   Thumb Code     0  llsdiv.o(.text)
    __2printf                                0x00000275   Thumb Code    22  noretval__2printf.o(.text)
    __2sprintf                               0x00000291   Thumb Code    36  noretval__2sprintf.o(.text)
    _printf_pre_padding                      0x000002b9   Thumb Code    44  _printf_pad.o(.text)
    _printf_post_padding                     0x000002e5   Thumb Code    34  _printf_pad.o(.text)
    _printf_str                              0x00000307   Thumb Code    82  _printf_str.o(.text)
    _printf_int_dec                          0x00000359   Thumb Code    90  _printf_dec.o(.text)
    _printf_int_hex                          0x000003c5   Thumb Code    84  _printf_hex_int.o(.text)
    _printf_longlong_hex                     0x000003c5   Thumb Code     0  _printf_hex_int.o(.text)
    __printf                                 0x0000041d   Thumb Code   306  __printf_flags_wp.o(.text)
    strlen                                   0x00000555   Thumb Code    62  strlen.o(.text)
    __aeabi_uidiv                            0x00000599   Thumb Code     0  aeabi_sdiv.o(.text)
    __aeabi_uidivmod                         0x00000599   Thumb Code    20  aeabi_sdiv.o(.text)
    __aeabi_idiv                             0x000005ad   Thumb Code     0  aeabi_sdiv.o(.text)
    __aeabi_idivmod                          0x000005ad   Thumb Code   326  aeabi_sdiv.o(.text)
    __use_two_region_memory                  0x000006f3   Thumb Code     2  heapauxi.o(.text)
    __rt_heap_escrow$2region                 0x000006f5   Thumb Code     2  heapauxi.o(.text)
    __rt_heap_expand$2region                 0x000006f7   Thumb Code     2  heapauxi.o(.text)
    __aeabi_uldivmod                         0x000006f9   Thumb Code   258  lludiv.o(.text)
    _ll_udiv                                 0x000006f9   Thumb Code     0  lludiv.o(.text)
    _printf_int_common                       0x000007fb   Thumb Code   176  _printf_intcommon.o(.text)
    _printf_char_common                      0x000008b7   Thumb Code    32  _printf_char_common.o(.text)
    _sputc                                   0x000008dd   Thumb Code    10  _sputc.o(.text)
    _printf_cs_common                        0x000008e7   Thumb Code    22  _printf_char.o(.text)
    _printf_char                             0x000008fd   Thumb Code    16  _printf_char.o(.text)
    _printf_string                           0x0000090d   Thumb Code     8  _printf_char.o(.text)
    _printf_char_file                        0x00000915   Thumb Code    34  _printf_char_file.o(.text)
    __rt_udiv10                              0x0000093d   Thumb Code    40  rtudiv10.o(.text)
    __user_libspace                          0x00000965   Thumb Code     8  libspace.o(.text)
    __user_perproc_libspace                  0x00000965   Thumb Code     0  libspace.o(.text)
    __user_perthread_libspace                0x00000965   Thumb Code     0  libspace.o(.text)
    __user_setup_stackheap                   0x0000096d   Thumb Code    62  sys_stackheap_outer.o(.text)
    exit                                     0x000009ab   Thumb Code    16  exit.o(.text)
    _sys_exit                                0x000009bd   Thumb Code     8  sys_exit.o(.text)
    __I$use$semihosting                      0x000009c9   Thumb Code     0  use_no_semi.o(.text)
    __use_no_semihosting_swi                 0x000009c9   Thumb Code     2  use_no_semi.o(.text)
    __semihosting_library_function           0x000009cb   Thumb Code     0  indicate_semi.o(.text)
    CLK_EnableModuleClock                    0x000009cd   Thumb Code    32  clk.o(i.CLK_EnableModuleClock)
    CLK_EnableXtalRC                         0x000009f1   Thumb Code    72  clk.o(i.CLK_EnableXtalRC)
    CLK_SetHCLK                              0x00000a3d   Thumb Code    94  clk.o(i.CLK_SetHCLK)
    CLK_SetModuleClock                       0x00000aa1   Thumb Code    94  clk.o(i.CLK_SetModuleClock)
    CLK_WaitClockReady                       0x00000b05   Thumb Code    32  clk.o(i.CLK_WaitClockReady)
    GPIO_SetMode                             0x00000b2d   Thumb Code    46  gpio.o(i.GPIO_SetMode)
    Hard_Fault_Handler                       0x00000b5d   Thumb Code    18  retarget.o(i.Hard_Fault_Handler)
    SendChar                                 0x00000b89   Thumb Code    12  retarget.o(i.SendChar)
    SendChar_ToUART                          0x00000b95   Thumb Code    48  retarget.o(i.SendChar_ToUART)
    SysGet_HCLKFreq                          0x00000bc9   Thumb Code    68  system_nano100series.o(i.SysGet_HCLKFreq)
    SysGet_PLLClockFreq                      0x00000c19   Thumb Code   120  system_nano100series.o(i.SysGet_PLLClockFreq)
    SystemCoreClockUpdate                    0x00000c99   Thumb Code    30  system_nano100series.o(i.SystemCoreClockUpdate)
    TIMER_Delay                              0x00000cc5   Thumb Code   168  timer.o(i.TIMER_Delay)
    TIMER_GetModuleClock                     0x00000d79   Thumb Code   102  timer.o(i.TIMER_GetModuleClock)
    UART1_IRQHandler                         0x00000df9   Thumb Code    20  main.o(i.UART1_IRQHandler)
    UART_ClearIntFlag                        0x00000e15   Thumb Code   112  uart.o(i.UART_ClearIntFlag)
    UART_EnableInt                           0x00000e85   Thumb Code     8  uart.o(i.UART_EnableInt)
    UART_Open                                0x00000e8d   Thumb Code   146  uart.o(i.UART_Open)
    UART_Write                               0x00000f2d   Thumb Code    54  uart.o(i.UART_Write)
    __ARM_common_ll_muluu                    0x00000f63   Thumb Code    48  timer.o(i.__ARM_common_ll_muluu)
    _is_digit                                0x00000f93   Thumb Code    14  __printf_wp.o(i._is_digit)
    ferror                                   0x00000fa1   Thumb Code     8  retarget.o(i.ferror)
    fputc                                    0x00000fa9   Thumb Code    16  retarget.o(i.fputc)
    init                                     0x00000fb9   Thumb Code   186  main.o(i.init)
    main                                     0x00001081   Thumb Code   266  main.o(i.main)
    stackDump                                0x000011fd   Thumb Code    70  retarget.o(i.stackDump)
    Region$$Table$$Base                      0x00001364   Number         0  anon$$obj.o(Region$$Table)
    Region$$Table$$Limit                     0x00001384   Number         0  anon$$obj.o(Region$$Table)
    __stdout                                 0x20000000   Data           4  retarget.o(.data)
    __stdin                                  0x20000004   Data           4  retarget.o(.data)
    SystemCoreClock                          0x20000008   Data           4  system_nano100series.o(.data)
    CyclesPerUs                              0x2000000c   Data           4  system_nano100series.o(.data)
    __libspace_start                         0x20000010   Data          96  libspace.o(.bss)
    __temporary_stack_top$libspace           0x20000070   Data           0  libspace.o(.bss)



==============================================================================

Memory Map of the image

  Image Entry point : 0x000000c1

  Load Region LR_IROM1 (Base: 0x00000000, Size: 0x00001394, Max: 0x00008000, ABSOLUTE)

    Execution Region ER_IROM1 (Base: 0x00000000, Size: 0x00001384, Max: 0x00008000, ABSOLUTE)

    Base Addr    Size         Type   Attr      Idx    E Section Name        Object

    0x00000000   0x000000c0   Data   RO          752    RESET               startup_nano100series.o
    0x000000c0   0x00000008   Code   RO          831  * !!!main             c_p.l(__main.o)
    0x000000c8   0x0000003c   Code   RO         1054    !!!scatter          c_p.l(__scatter.o)
    0x00000104   0x0000001a   Code   RO         1056    !!handler_copy      c_p.l(__scatter_copy.o)
    0x0000011e   0x00000002   PAD
    0x00000120   0x0000001c   Code   RO         1058    !!handler_zi        c_p.l(__scatter_zi.o)
    0x0000013c   0x00000002   Code   RO          822    .ARM.Collect$$_printf_percent$$00000000  c_p.l(_printf_percent.o)
    0x0000013e   0x0000000a   Code   RO          820    .ARM.Collect$$_printf_percent$$00000009  c_p.l(_printf_d.o)
    0x00000148   0x0000000a   Code   RO          819    .ARM.Collect$$_printf_percent$$0000000C  c_p.l(_printf_x.o)
    0x00000152   0x0000000a   Code   RO          818    .ARM.Collect$$_printf_percent$$00000014  c_p.l(_printf_s.o)
    0x0000015c   0x00000004   Code   RO          861    .ARM.Collect$$_printf_percent$$00000017  c_p.l(_printf_percent_end.o)
    0x00000160   0x00000002   Code   RO          928    .ARM.Collect$$libinit$$00000000  c_p.l(libinit.o)
    0x00000162   0x00000000   Code   RO          930    .ARM.Collect$$libinit$$00000002  c_p.l(libinit2.o)
    0x00000162   0x00000000   Code   RO          932    .ARM.Collect$$libinit$$00000004  c_p.l(libinit2.o)
    0x00000162   0x00000000   Code   RO          935    .ARM.Collect$$libinit$$0000000A  c_p.l(libinit2.o)
    0x00000162   0x00000000   Code   RO          937    .ARM.Collect$$libinit$$0000000C  c_p.l(libinit2.o)
    0x00000162   0x00000000   Code   RO          939    .ARM.Collect$$libinit$$0000000E  c_p.l(libinit2.o)
    0x00000162   0x00000000   Code   RO          942    .ARM.Collect$$libinit$$00000011  c_p.l(libinit2.o)
    0x00000162   0x00000000   Code   RO          944    .ARM.Collect$$libinit$$00000013  c_p.l(libinit2.o)
    0x00000162   0x00000000   Code   RO          946    .ARM.Collect$$libinit$$00000015  c_p.l(libinit2.o)
    0x00000162   0x00000000   Code   RO          948    .ARM.Collect$$libinit$$00000017  c_p.l(libinit2.o)
    0x00000162   0x00000000   Code   RO          950    .ARM.Collect$$libinit$$00000019  c_p.l(libinit2.o)
    0x00000162   0x00000000   Code   RO          952    .ARM.Collect$$libinit$$0000001B  c_p.l(libinit2.o)
    0x00000162   0x00000000   Code   RO          954    .ARM.Collect$$libinit$$0000001D  c_p.l(libinit2.o)
    0x00000162   0x00000000   Code   RO          956    .ARM.Collect$$libinit$$0000001F  c_p.l(libinit2.o)
    0x00000162   0x00000000   Code   RO          958    .ARM.Collect$$libinit$$00000021  c_p.l(libinit2.o)
    0x00000162   0x00000000   Code   RO          960    .ARM.Collect$$libinit$$00000023  c_p.l(libinit2.o)
    0x00000162   0x00000000   Code   RO          962    .ARM.Collect$$libinit$$00000025  c_p.l(libinit2.o)
    0x00000162   0x00000000   Code   RO          966    .ARM.Collect$$libinit$$0000002C  c_p.l(libinit2.o)
    0x00000162   0x00000000   Code   RO          968    .ARM.Collect$$libinit$$0000002E  c_p.l(libinit2.o)
    0x00000162   0x00000000   Code   RO          970    .ARM.Collect$$libinit$$00000030  c_p.l(libinit2.o)
    0x00000162   0x00000000   Code   RO          972    .ARM.Collect$$libinit$$00000032  c_p.l(libinit2.o)
    0x00000162   0x00000002   Code   RO          973    .ARM.Collect$$libinit$$00000033  c_p.l(libinit2.o)
    0x00000164   0x00000002   Code   RO         1019    .ARM.Collect$$libshutdown$$00000000  c_p.l(libshutdown.o)
    0x00000166   0x00000000   Code   RO         1037    .ARM.Collect$$libshutdown$$00000002  c_p.l(libshutdown2.o)
    0x00000166   0x00000000   Code   RO         1039    .ARM.Collect$$libshutdown$$00000004  c_p.l(libshutdown2.o)
    0x00000166   0x00000000   Code   RO         1042    .ARM.Collect$$libshutdown$$00000007  c_p.l(libshutdown2.o)
    0x00000166   0x00000000   Code   RO         1045    .ARM.Collect$$libshutdown$$0000000A  c_p.l(libshutdown2.o)
    0x00000166   0x00000000   Code   RO         1047    .ARM.Collect$$libshutdown$$0000000C  c_p.l(libshutdown2.o)
    0x00000166   0x00000000   Code   RO         1050    .ARM.Collect$$libshutdown$$0000000F  c_p.l(libshutdown2.o)
    0x00000166   0x00000002   Code   RO         1051    .ARM.Collect$$libshutdown$$00000010  c_p.l(libshutdown2.o)
    0x00000168   0x00000000   Code   RO          842    .ARM.Collect$$rtentry$$00000000  c_p.l(__rtentry.o)
    0x00000168   0x00000000   Code   RO          866    .ARM.Collect$$rtentry$$00000002  c_p.l(__rtentry2.o)
    0x00000168   0x00000006   Code   RO          878    .ARM.Collect$$rtentry$$00000004  c_p.l(__rtentry4.o)
    0x0000016e   0x00000000   Code   RO          868    .ARM.Collect$$rtentry$$00000009  c_p.l(__rtentry2.o)
    0x0000016e   0x00000004   Code   RO          869    .ARM.Collect$$rtentry$$0000000A  c_p.l(__rtentry2.o)
    0x00000172   0x00000000   Code   RO          871    .ARM.Collect$$rtentry$$0000000C  c_p.l(__rtentry2.o)
    0x00000172   0x00000008   Code   RO          872    .ARM.Collect$$rtentry$$0000000D  c_p.l(__rtentry2.o)
    0x0000017a   0x00000002   Code   RO          975    .ARM.Collect$$rtexit$$00000000  c_p.l(rtexit.o)
    0x0000017c   0x00000000   Code   RO          990    .ARM.Collect$$rtexit$$00000002  c_p.l(rtexit2.o)
    0x0000017c   0x00000004   Code   RO          991    .ARM.Collect$$rtexit$$00000003  c_p.l(rtexit2.o)
    0x00000180   0x00000006   Code   RO          992    .ARM.Collect$$rtexit$$00000004  c_p.l(rtexit2.o)
    0x00000186   0x00000002   PAD
    0x00000188   0x0000001c   Code   RO          275    .emb_text           retarget.o
    0x000001a4   0x00000060   Code   RO          753    .text               startup_nano100series.o
    0x00000204   0x00000070   Code   RO          759    .text               c_p.l(llsdiv.o)
    0x00000274   0x0000001c   Code   RO          765    .text               c_p.l(noretval__2printf.o)
    0x00000290   0x00000028   Code   RO          767    .text               c_p.l(noretval__2sprintf.o)
    0x000002b8   0x0000004e   Code   RO          771    .text               c_p.l(_printf_pad.o)
    0x00000306   0x00000052   Code   RO          773    .text               c_p.l(_printf_str.o)
    0x00000358   0x0000006c   Code   RO          775    .text               c_p.l(_printf_dec.o)
    0x000003c4   0x00000058   Code   RO          780    .text               c_p.l(_printf_hex_int.o)
    0x0000041c   0x00000138   Code   RO          810    .text               c_p.l(__printf_flags_wp.o)
    0x00000554   0x00000044   Code   RO          823    .text               c_p.l(strlen.o)
    0x00000598   0x0000015a   Code   RO          825    .text               c_p.l(aeabi_sdiv.o)
    0x000006f2   0x00000006   Code   RO          829    .text               c_p.l(heapauxi.o)
    0x000006f8   0x00000102   Code   RO          847    .text               c_p.l(lludiv.o)
    0x000007fa   0x000000b0   Code   RO          849    .text               c_p.l(_printf_intcommon.o)
    0x000008aa   0x00000002   PAD
    0x000008ac   0x00000030   Code   RO          853    .text               c_p.l(_printf_char_common.o)
    0x000008dc   0x0000000a   Code   RO          855    .text               c_p.l(_sputc.o)
    0x000008e6   0x0000002e   Code   RO          857    .text               c_p.l(_printf_char.o)
    0x00000914   0x00000028   Code   RO          859    .text               c_p.l(_printf_char_file.o)
    0x0000093c   0x00000028   Code   RO          862    .text               c_p.l(rtudiv10.o)
    0x00000964   0x00000008   Code   RO          909    .text               c_p.l(libspace.o)
    0x0000096c   0x0000003e   Code   RO          912    .text               c_p.l(sys_stackheap_outer.o)
    0x000009aa   0x00000010   Code   RO          915    .text               c_p.l(exit.o)
    0x000009ba   0x00000002   PAD
    0x000009bc   0x0000000c   Code   RO          987    .text               c_p.l(sys_exit.o)
    0x000009c8   0x00000002   Code   RO         1006    .text               c_p.l(use_no_semi.o)
    0x000009ca   0x00000000   Code   RO         1008    .text               c_p.l(indicate_semi.o)
    0x000009ca   0x00000002   PAD
    0x000009cc   0x00000024   Code   RO            9    i.CLK_EnableModuleClock  clk.o
    0x000009f0   0x0000004c   Code   RO           12    i.CLK_EnableXtalRC  clk.o
    0x00000a3c   0x00000064   Code   RO           21    i.CLK_SetHCLK       clk.o
    0x00000aa0   0x00000064   Code   RO           22    i.CLK_SetModuleClock  clk.o
    0x00000b04   0x00000028   Code   RO           24    i.CLK_WaitClockReady  clk.o
    0x00000b2c   0x0000002e   Code   RO          245    i.GPIO_SetMode      gpio.o
    0x00000b5a   0x00000002   PAD
    0x00000b5c   0x0000002c   Code   RO          277    i.Hard_Fault_Handler  retarget.o
    0x00000b88   0x0000000c   Code   RO          279    i.SendChar          retarget.o
    0x00000b94   0x00000034   Code   RO          280    i.SendChar_ToUART   retarget.o
    0x00000bc8   0x00000050   Code   RO          714    i.SysGet_HCLKFreq   system_nano100series.o
    0x00000c18   0x00000080   Code   RO          715    i.SysGet_PLLClockFreq  system_nano100series.o
    0x00000c98   0x0000002c   Code   RO          716    i.SystemCoreClockUpdate  system_nano100series.o
    0x00000cc4   0x000000b4   Code   RO          478    i.TIMER_Delay       timer.o
    0x00000d78   0x00000080   Code   RO          485    i.TIMER_GetModuleClock  timer.o
    0x00000df8   0x0000001c   Code   RO          669    i.UART1_IRQHandler  main.o
    0x00000e14   0x00000070   Code   RO          570    i.UART_ClearIntFlag  uart.o
    0x00000e84   0x00000008   Code   RO          575    i.UART_EnableInt    uart.o
    0x00000e8c   0x000000a0   Code   RO          576    i.UART_Open         uart.o
    0x00000f2c   0x00000036   Code   RO          583    i.UART_Write        uart.o
    0x00000f62   0x00000030   Code   RO          559    i.__ARM_common_ll_muluu  timer.o
    0x00000f92   0x0000000e   Code   RO          808    i._is_digit         c_p.l(__printf_wp.o)
    0x00000fa0   0x00000008   Code   RO          282    i.ferror            retarget.o
    0x00000fa8   0x00000010   Code   RO          284    i.fputc             retarget.o
    0x00000fb8   0x000000c8   Code   RO          670    i.init              main.o
    0x00001080   0x0000017c   Code   RO          671    i.main              main.o
    0x000011fc   0x000000a8   Code   RO          286    i.stackDump         retarget.o
    0x000012a4   0x00000010   Data   RO          489    .constdata          timer.o
    0x000012b4   0x00000030   Data   RO          584    .constdata          uart.o
    0x000012e4   0x00000028   Data   RO          781    .constdata          c_p.l(_printf_hex_int.o)
    0x0000130c   0x00000011   Data   RO          811    .constdata          c_p.l(__printf_flags_wp.o)
    0x0000131d   0x00000003   PAD
    0x00001320   0x00000043   Data   RO          672    .conststring        main.o
    0x00001363   0x00000001   PAD
    0x00001364   0x00000020   Data   RO         1052    Region$$Table       anon$$obj.o


    Execution Region RW_IRAM1 (Base: 0x20000000, Size: 0x00000a70, Max: 0x00002000, ABSOLUTE)

    Base Addr    Size         Type   Attr      Idx    E Section Name        Object

    0x20000000   0x00000008   Data   RW          287    .data               retarget.o
    0x20000008   0x00000008   Data   RW          717    .data               system_nano100series.o
    0x20000010   0x00000060   Zero   RW          910    .bss                c_p.l(libspace.o)
    0x20000070   0x00000500   Zero   RW          751    HEAP                startup_nano100series.o
    0x20000570   0x00000500   Zero   RW          750    STACK               startup_nano100series.o


==============================================================================

Image component sizes


      Code (inc. data)   RO Data    RW Data    ZI Data      Debug   Object Name

       352         28          0          0          0     118915   clk.o
        46          0          0          0          0        971   gpio.o
       608        136         67          0          0      36449   main.o
       328        132          0          8          0     116829   retarget.o
        96         46        192          0       2560        744   startup_nano100series.o
       252         34          0          8          0       2462   system_nano100series.o
       356         38         16          0          0       2017   timer.o
       334         14         48          0          0       3134   uart.o

    ----------------------------------------------------------------------
      2374        428        356         16       2560     281521   Object Totals
         0          0         32          0          0          0   (incl. Generated)
         2          0          1          0          0          0   (incl. Padding)

    ----------------------------------------------------------------------

      Code (inc. data)   RO Data    RW Data    ZI Data      Debug   Library Member Name

         8          0          0          0          0         68   __main.o
       312          6         17          0          0         76   __printf_flags_wp.o
        14          0          0          0          0         60   __printf_wp.o
         0          0          0          0          0          0   __rtentry.o
        12          0          0          0          0          0   __rtentry2.o
         6          0          0          0          0          0   __rtentry4.o
        60          8          0          0          0          0   __scatter.o
        26          0          0          0          0          0   __scatter_copy.o
        28          0          0          0          0          0   __scatter_zi.o
        46          0          0          0          0        100   _printf_char.o
        48          6          0          0          0         88   _printf_char_common.o
        40          6          0          0          0         72   _printf_char_file.o
        10          0          0          0          0          0   _printf_d.o
       108         18          0          0          0         76   _printf_dec.o
        88          4         40          0          0         72   _printf_hex_int.o
       176          0          0          0          0         84   _printf_intcommon.o
        78          0          0          0          0        100   _printf_pad.o
         2          0          0          0          0          0   _printf_percent.o
         4          0          0          0          0          0   _printf_percent_end.o
        10          0          0          0          0          0   _printf_s.o
        82          0          0          0          0         72   _printf_str.o
        10          0          0          0          0          0   _printf_x.o
        10          0          0          0          0         60   _sputc.o
       346          0          0          0          0         92   aeabi_sdiv.o
        16          0          0          0          0         68   exit.o
         6          0          0          0          0        136   heapauxi.o
         0          0          0          0          0          0   indicate_semi.o
         2          0          0          0          0          0   libinit.o
         2          0          0          0          0          0   libinit2.o
         2          0          0          0          0          0   libshutdown.o
         2          0          0          0          0          0   libshutdown2.o
         8          4          0          0         96         68   libspace.o
       112          0          0          0          0         72   llsdiv.o
       258          0          0          0          0         88   lludiv.o
        28          6          0          0          0         84   noretval__2printf.o
        40          4          0          0          0         84   noretval__2sprintf.o
         2          0          0          0          0          0   rtexit.o
        10          0          0          0          0          0   rtexit2.o
        40          0          0          0          0         60   rtudiv10.o
        68          6          0          0          0         72   strlen.o
        12          4          0          0          0         60   sys_exit.o
        62          0          0          0          0         80   sys_stackheap_outer.o
         2          0          0          0          0         68   use_no_semi.o

    ----------------------------------------------------------------------
      2206         72         60          0         96       1960   Library Totals
        10          0          3          0          0          0   (incl. Padding)

    ----------------------------------------------------------------------

      Code (inc. data)   RO Data    RW Data    ZI Data      Debug   Library Name

      2196         72         57          0         96       1960   c_p.l

    ----------------------------------------------------------------------
      2206         72         60          0         96       1960   Library Totals

    ----------------------------------------------------------------------

==============================================================================


      Code (inc. data)   RO Data    RW Data    ZI Data      Debug   

      4580        500        416         16       2656     281525   Grand Totals
      4580        500        416         16       2656     281525   ELF Image Totals
      4580        500        416         16          0          0   ROM Totals

==============================================================================

    Total RO  Size (Code + RO Data)                 4996 (   4.88kB)
    Total RW  Size (RW Data + ZI Data)              2672 (   2.61kB)
    Total ROM Size (Code + RO Data + RW Data)       5012 (   4.89kB)

==============================================================================

